:100000000C94F3020C941B030C941B030C941B0321
:100010000C941B030C941B030C941B030C941B03E8
:100020000C941B030C941B030C941B030C94A92D20
:100030000C941B030C941B030C941B030C941B03C8
:100040000C940F2E0C941B030C941B030C941B0399
:100050000C941B030C941B030C941B030C941B03A8
:100060000C941B030C941B034572726F7200476162
:100070006D65206C6F6164656400536176696E67BD
:100080002067616D65004E6F7468696E6720746FDC
:1000900020626520736176656421004E6F20736174
:1000A0007665642067616D650046696C6520656DE5
:1000B000707479004C6F6164696E67207361766556
:1000C000642067616D6500436C65616E696E6720D1
:1000D000454550524F4D00202D204E6F20646573D2
:1000E0006372697074696F6E202D20001120444581
:1000F0004C4554452047414D4520100011204445B2
:100100004C45544520534156452010001120504C79
:100110004159201000486F6C64204120746F2064A6
:10012000656C65746500202120444F4E275420548F
:1001300055524E204F46462021200020201D204CA5
:100140006F6164696E672067616D652E2E2E2020B9
:1001500000496E73657274205344202620726573C3
:1001600074617274001D2052656164696E6720536A
:100170004420636172642E2E2E0A0A000808CACB3E
:10018000C3FF818181FF40240000000000000000C7
:10019000000000000000000000000000000000005F
:1001A00000000001F8FFFFFC00000003F9FFFFFE64
:1001B00000000007FFFFFFFF000007FFFFFFFFFF3A
:1001C00000000FFF0330C71F00001C060120820F34
:1001D00000001C0649E7924F00001FFE49279E4F72
:1001E00000001C0649279E4F00001C0679209E0F28
:1001F00000001FFE79309F1F00001C0679FFFFFFE3
:1002000000001C07FF0041BF00001FFFFC00466FFD
:1002100000001807F87FFD8700001807FC0FFE0399
:1002200000001FFFFE03FE0300001C07FFC1800744
:1002300000001C07F001801F00001FFFE003007F8B
:1002400000001807E00F07FF00001807FFFFFFFF7F
:1002500000001FFFFFFFFFFF00001C07FF7FFBFFE9
:1002600000001C07FF77337300001FFFFF6AAAAF6F
:1002700000001C07FF6AAA6F00001C07FFB7332F9E
:1002800000000FFFFFFFFFFE000007FFFFFFFFFC66
:10029000000000000000000000000000000000005E
:1002A00000000000000000000A4E6F20534420634D
:1002B000617264206F720A6E6F204C4F4144455248
:1002C0002E4845580A0A153A45786974001D20469B
:1002D0006C617368696E670A20206C6F6164657277
:1002E0002E2E2E0A0A444F4E2754205455524E208B
:1002F0004F464621000A0A153A49676E6F7265003B
:100300006D560A0A504C45415345205455524E20D3
:100310004F464620004C4F572042415454455259B5
:10032000212000172B152010204C4F41444552002E
:10033000172B1620131400175344001613780016B9
:10034000131400151020001520100000540A03E1BA
:1003500081867F3E186D830F0F0E018386603318F0
:100360006DC3198F1803C38E6033186DE330CF1837
:1003700003C39E603630CDE360CF3006C79E7E3E1D
:1003800030CDB360CF300CC6F6603330D9B660CF15
:1003900033CFCCF66061B0DB1E60CF30D86CE6C0E6
:1003A00061B0DB1E618F19986CC6C063B19B0E33C0
:1003B0000F0FB078C6FF7E1F1B061E0F0500893089
:1003C0000802380249786814000003053F213F12F3
:1003D00008120A100A0E1C0E0C1E0C141A14161FFA
:1003E000161E131E1E1B1E1E1F1E3F213F3A2F3AB4
:1003F000173D173F213F181F02040A041F0E040473
:100400000E1F0A1F0A0E0E1F04110E2E252E2F2A54
:100410002E262929021F02081F08150E04040E1596
:100420000E15151B151B040604040C040000000027
:1004300017000300031F0A1F16371A1904130A15A1
:100440003A000300000E11110E000A040A040E0403
:100450000030000404040010001804031F111F12D0
:100460001F101D151711151F07041F17151D1F1528
:100470001D01011F1F151F17151F000A0000320064
:10048000040A110A0A0A110A040115020E11171EA4
:10049000051E1F150A0E110A1F110E1F15111F052B
:1004A000010E111D1F041F111F1108100F1F041B27
:1004B0001F10101F061F1E040F0E110E1F09060E1F
:1004C000112E1F051A121509011F011F101F0F18E9
:1004D0000F1F0C1F1B041B031C03191513001F11F6
:1004E000030418111F000201022020200001020C49
:1004F000121E1F120C0C12120C121F0C1A14041EC6
:1005000005242A1E1F021C141D1020201D1F081464
:10051000111F101E041E1E021C0C120C3E0A040C9D
:10052000123E1E040214160A020F120E101E0E10A6
:100530000E1E081E120C1226281E322A26041E2108
:10054000001F00211E040102013F213FF6E8DBCF1E
:10055000C3B8AEA49B928A827B746E68625C575269
:100560004E4945413E3A3734312E2C292725232147
:10057000450068010000050038016801000086059B
:1005800082050101FF030101F703000000080002DA
:100590000100000304070000000000000000010249
:1005A0000408102040800102040810200102040801
:1005B00010200404040404040404020202020202DF
:1005C00003030303030300000000230026002900A7
:1005D00000000000250028002B000000000024007F
:1005E00027002A00BC0D11241FBECFEFD8E0DEBFCC
:1005F000CDBF11E0A0E0B1E0E6EBF7E602C0059068
:100600000D92A436B107D9F727E0A4E6B1E001C006
:100610001D92AB35B207E1F715E0C6EED5E004C098
:100620002297FE010E945F33C43ED107C9F70E94A2
:10063000A0310C94D9330C940000FB0105900020EC
:10064000E9F7609570956E0F7F1FCB0108950496B2
:100650000C943315895B9D4F0C94840F895B9D4FDF
:100660000C94EB0FCF93DF931F92CDB7DEB7698366
:1006700041E050E0BE016F5F7F4F04960E9433154A
:100680000F90DF91CF910895FB01242F60914905D0
:1006900070914A05AF010C94AE14FF920F931F9313
:1006A000CF93DF938C01F62EEC01C95DDD4FCE01B7
:1006B0000E94A514B801CE010E94F610882359F0BB
:1006C000FF2039F08881807731F0D0934A05C093BC
:1006D000490581E001C080E0DF91CF911F910F912A
:1006E000FF900895DC01643508F053C0403308F0F2
:1006F00050C090968C919097342F359535953595BF
:10070000E62FFF27E7FDF095242F2770823099F41C
:10071000DF01A45BBA4F84E53802A00DB11D11249E
:100720008C9190E0022E02C0959587950A94E2F78D
:100730008095817009C0833039F446271C968C91CE
:10074000482740FF03C014C0811112C084E538025D
:10075000E00DF11D1124E45BFA4F81E090E0022EE0
:1007600001C0880F0A94EAF780959081982310C001
:1007700084E53802E00DF11D1124E45BFA4F81E0BD
:1007800090E0022E01C0880F0A94EAF79081982B1E
:1007900090830895A9E6B1E0E0E8F7E784918D93AE
:1007A0003196E11588E7F807C9F7E4E4F2E0ABE633
:1007B000B1E081918D9382E0ED34F807D1F769E6DD
:1007C00071E080E897E7EDEFFFE309940F9361E0B4
:1007D0008EE095E00E94132607E024E540E060E00B
:1007E0008EE095E00E94892682E08093170581E0E3
:1007F0008093180560E08EE095E00E94132601E0EA
:1008000024E547E060E08EE095E00E9489260F91A4
:1008100008950F9361E08EE095E00E94132607E0B3
:1008200024E549E260E08EE095E00E94892682E0BE
:10083000809317058AE28093180560E08EE095E0CA
:100840000E94132601E024E548E260E08EE095E096
:100850000E9489260F910895CF93DF93EC01BC018C
:10086000882777FD8095982F0E941D0320911605FB
:1008700040911205429FA0011124489F9001499F79
:10088000300D589F300D1124369527958AE2821B32
:1008900080931705BE018EE095E0DF91CF910C9417
:1008A0006230CF93DF9300D0CDB7DEB789839A83D0
:1008B0000E94E60389819A810F900F90DF91CF917A
:1008C0000C942C04CF93DF9300D0CDB7DEB789838F
:1008D0009A830E94090489819A810F900F90DF9179
:1008E000CF910C942C04FC0101900020E9F7319782
:1008F000E81BF90B2091160540911205429FA001BB
:1009000011244E9F90014F9F300D5E9F300D11249A
:10091000369527953AE2321B30931705BC018EE0DD
:1009200095E00C948530CF93DF9300D0CDB7DEB740
:1009300089839A830E94E60389819A810F900F90A0
:10094000DF91CF910C947304CF93DF9300D0CDB798
:10095000DEB789839A830E94090489819A810F9066
:100960000F90DF91CF910C9473042F923F924F928E
:100970005F926F927F928F929F92AF92BF92CF922F
:10098000DF92EF92FF920F931F93CF93DF9300D0EC
:1009900000D0CDB7DEB7582E662E742E422EB80189
:1009A00041E081E592E00E944403882309F481C07C
:1009B000472D50E0495F5F4F63E0559547956A9535
:1009C000E1F75C834B835B81598380E890E06B8126
:1009D0007C810E94FD326B016A83A70160E070E0B8
:1009E00081E592E00E94A21200E010E0A42CB12C5C
:1009F00070E8872E912C202E041508F054C0822D0B
:100A00006A810E94DD32392E992371F08B819C819D
:100A1000389E7001399EF00C1124312CF701E759F2
:100A2000FE4F7F01260C3AC07501E01AF10ACE1480
:100A3000DF040CF47601F981FE9DE02C1124F12CE9
:100A4000A70169E671E081E592E00E9410118E1520
:100A50009F05E4F681E592E00E94A5142AC0832D4B
:100A6000869586958695F701E80FF11D8081992777
:100A700087FD9095232D2770A40102C055954795B9
:100A80002A95E2F784239523892B39F0422D632D93
:100A9000650D8EE095E00E94720333943710DFCF2E
:100AA0000F5F1F4FA8CF81E592E00E94A51481E05F
:100AB00001C080E00F900F900F900F90DF91CF91C9
:100AC0001F910F91FF90EF90DF90CF90BF90AF906C
:100AD0009F908F907F906F905F904F903F902F905E
:100AE0000895EF92FF920F931F93CF93DF93EC0142
:100AF00060E08EE095E00E94132600E224E548E0E5
:100B000060E08EE095E00E94892661E08EE095E04D
:100B10000E9413266091F30189E0689FB0011124BF
:100B20006C507E4F8FE091E00E9493336EE171E054
:100B30008FE091E00E94883380E691E0C89F7001C9
:100B4000C99FF00CD89FF00C112481E5E80EF11C30
:100B50000FE011E020E244E568E080E00E94B50487
:100B6000DF91CF911F910F91FF90EF900895CF9358
:100B70008EE095E00E94BA2561E08EE095E00E944B
:100B8000132610926801109267018EE18093640130
:100B900010926601109265016091F30189E0689FEF
:100BA000B00111246C507E4F8FE091E00E9493338E
:100BB0006EE171E08FE091E00E94883341E06FE0E8
:100BC00071E081E592E00E944403882389F141E5C8
:100BD00050E069E671E081E592E00E9410118135F4
:100BE000910531F580916F01813011F510928301EB
:100BF00080E791E00E9493048091B901809368019D
:100C000081E592E00E94A5148091670190E00E9426
:100C10007105811141C086E18093180583E08093BE
:100C2000170567ED70E08EE095E0CF910C9462308F
:100C30006091F301C9E0C69FB00111246C507E4F52
:100C40008FE091E00E94933369E271E08FE091E0E0
:100C50000E94883310927B0141E06FE071E081E5F2
:100C600092E00E94440380915402882359F042E1AB
:100C700050E069E671E081E592E00E94D81689E6CD
:100C800091E007C08091F301C89FC00111248C50EE
:100C90009E4F0E949304B4CFCF910895EFE0F1E00E
:100CA000A0E080E0811104C090819E32B1F405C0C3
:100CB000813021F490819E3281F08F5F823069F41F
:100CC00091E09A0FB0E0A351BE4F20812C93933056
:100CD00019F41092F0010895A92F319691E0EC31AA
:100CE000F90701F7F6CF6FE071E081E592E00E942D
:100CF0001E1C0E944E066AE271E08DEE91E00E9499
:100D0000A933892B69F063E271E08FE091E00E94E2
:100D1000A933892B29F490915102907781E009F051
:100D200080E008950F93482F4695469593E1499F9B
:100D3000402D1124837094E1899F602D112404E1DA
:100D400025E18EE095E00E9461260F9108950F93B2
:100D5000CF9361E08EE095E00E9413268091F2012E
:100D6000883010F40E94920660E08EE095E00E94C8
:100D700013268091F3010E9492066091F301609323
:100D8000F20189E0689FB00111246C507E4F8FE022
:100D900091E00E9493336EE171E08FE091E00E9458
:100DA000883341E06FE071E081E592E00E94440306
:100DB000882309F45AC041E550E069E671E081E515
:100DC00092E00E9410118135910509F04EC080918A
:100DD0006F01813009F049C01092830180E791E0F2
:100DE0000E94A40481E592E00E94A5146091F301A1
:100DF00089E0689FB00111246C507E4F8FE091E034
:100E00000E9493336EE271E08FE091E00E9488339C
:100E100041E06FE071E081E592E00E9444038823A5
:100E2000F1F081E592E00E94A51460E08EE095E08B
:100E30000E94132608E029E048E260E08EE095E099
:100E40000E94892661E08EE095E00E9413262CE73F
:100E500031E048E260E08EE095E00E94312885EEC6
:100E600094E0CF910F910C94E32D6091F301C9E0D0
:100E7000C69FB00111246C507E4F8FE091E00E941C
:100E8000933369E271E08FE091E00E948833109221
:100E90007B0141E06FE071E081E592E00E94440354
:100EA00080915402882359F042E150E069E671E0F4
:100EB00081E592E00E94D81689E691E091CF809179
:100EC000F301C89FC00111248C509E4F89CF8F928F
:100ED0009F92AF92BF92CF92DF92EF92FF920F93C9
:100EE0001F93CF93DF938EE095E00E94BA2561E0D7
:100EF0008EE095E00E941326C0E027E240E06C2FD0
:100F00008EE095E00E941B26CC5EC837B1F7C0E0AA
:100F100020E54C2F60E08EE095E00E943E26CD5EFD
:100F2000CC34B1F761E081E792E00E944D0310926A
:100F3000F101C0E0D0E019E041E068E974E081E54A
:100F400092E00E94ED13882309F44FC00E947306BB
:100F5000882309F445C04091F10141110DC08091F1
:100F60003E0290913F029E0103E0359527950A9538
:100F7000E1F72817390799F5EFE0F1E089E0489F9C
:100F8000900111242C503E4F80E090E0582F619149
:100F90006E3249F4FC01149FE00DF11D1124EC5058
:100FA000FE4F108209C0D901A80FB91F6C9301969A
:100FB0008830910559F758E05F5F149FF0011124C4
:100FC000E50FF11DEC50FE4F10824F5F4093F10191
:100FD000483030F081E592E00E94A51406C02196C9
:100FE00081E592E00E94A514A7CF61E08EE095E034
:100FF0000E9413268091400290914102029744F191
:1010000007E224E040E060E58EE095E00E94612682
:10101000209140023091410285E290E0B9010E94A6
:10102000FD3201E0060F40913E0250913F0265E221
:10103000649FC001659F900D1124B9010E94FD328B
:1010400041E0460F23E061E58EE095E00E948926AD
:101050004091F101242F30E08091F30190E082175C
:1010600093071CF041504093F301D12CF9E0AF2ECF
:10107000A4E19A2EB3E18B2E8091F101D81608F0ED
:1010800056C0AD9CE0011124CC50DE4FBE018FE074
:1010900091E00E9493336EE171E08FE091E00E9455
:1010A00088331D2D1370199DB02C1124CD2CC6949E
:1010B000C694C89CC02C112461E06C0DEAE1EE2EB0
:1010C000F12C0FE011E022E143E181E08B0D0E9461
:1010D000B50481112AC01B2D1D5F1093170582E0F6
:1010E0008C0D8093180544E050E0BE018AE091E049
:1010F0000E949A336AE071E08EE095E00E948530AC
:10110000109317058C2D885F80931805BE016C5FC6
:101110007F4F44E050E08AE091E00E949A336AE019
:1011200071E08EE095E00E948530D394A5CF88E0F1
:101130008093F201DF91CF911F910F91FF90EF907B
:10114000DF90CF90BF90AF909F908F900C94A706A8
:10115000CF93DF93EC0187EC90E00E9462048EE075
:1011600095E00E94CB25C11584E0D8075CF4CE0140
:101170000E94C333882321F060E0CE010E94CB336C
:101180002196F1CFDF91CF910895DF92EF92FF92F8
:101190000F931F93CF93DF9364E472E08FE091E0AD
:1011A0000E949333EFE0F1E08081803209F41082F5
:1011B000319681E0E731F807B9F76EE271E08FE030
:1011C00091E00E94883341E06FE071E081E592E0B8
:1011D0000E944403882309F440C084EB90E00E94FD
:1011E00062048EE095E00E94CB25D12CF12C40E8E2
:1011F00050E069E671E081E592E00E9410118C01F7
:10120000181619060CF5CD2DDF2DEC2EED18F12C4E
:10121000E016F1069CF5CE010E94C333F701E759B1
:10122000FE4F6081482F50E0262F332727FD309551
:101230004217530719F0CE010E94CB332196C115F6
:1012400084E0D80714F31AC02D2D3F2D232BC9F4A9
:1012500089EA90E00E94620414C08BE990E00E9449
:101260006204D12CF12C8D2D9F2DDF91CF911F91F8
:101270000F91FF90EF90DF900C94A808DC2EFD2ECC
:10128000B6CF81E592E00E94A514EDCF6091F30105
:1012900089E0689FB00111246C507E4F84E492E095
:1012A0000E9493330E94CA030E94C50880E090E028
:1012B0000E947105811107C084E18093180584E4C0
:1012C00092E00E9473048BE391E00E94510486E255
:1012D00091E00E9462048EE095E00E94CB2584E4B8
:1012E00092E0EEEFFFE30994BF92CF92DF92EF928C
:1012F000FF920F93CF93DF930E94B70589E0C82E2A
:10130000C3E0D0E092E2E92EF12CBB24B3942CE0B0
:10131000D22E80EC94E00E948B208823D1F365E0EC
:101320008AEC94E00E946825811107C066E08AEC8F
:1013300094E00E946825882359F085EE94E00E948D
:10134000E32D80916501882309F4BBC110926501EA
:1013500064E08AEC94E00E946825882399F085EE89
:1013600094E00E94E32D80916601813049F028F0DD
:10137000823041F4B092650105C00E94460902C066
:1013800080936501809165018823A1F144E164E0C7
:101390008AEC94E00E947125882361F185EE94E047
:1013A0000E94E32D809166018130C9F56091F301BF
:1013B000C69EB00111246C507E4F8FE091E00E94D8
:1013C00093336EE271E08FE091E00E94883343E056
:1013D0006FE071E081E592E00E944403882341F0D0
:1013E00081E592E00E94991881E592E00E94A5149F
:1013F0000E94B70561E08AEC94E00E9468258111A3
:1014000049C18091D2048B3008F45AC043E061E0B6
:101410008AEC94E00E947F2581113CC151C082304A
:1014200049F76091F30159E0659FB00111246C50B8
:101430007E4F8FE091E00E9493336EE171E08FE088
:1014400091E00E94883343E06FE071E081E592E033
:101450000E944403882341F081E592E00E9499189C
:1014600081E592E00E94A5146091F30189E0689FF4
:10147000B00111246C507E4F8FE091E00E949333B5
:1014800069E271E08FE091E00E94883343E06FE011
:1014900071E081E592E00E944403882309F411C1C0
:1014A00081E592E00E94991881E592E0DF91CF9169
:1014B0000F91FF90EF90DF90CF90BF900C94A51408
:1014C00063E08AEC94E00E9468258111EAC0809173
:1014D000D4048B3040F043E063E08AEC94E00E9457
:1014E0007F258111DEC043E062E08AEC94E00E9437
:1014F0007F25882329F08091660190E001960CC039
:1015000043E060E08AEC94E00E947F25882349F064
:101510008091660190E00296BE010E94FD328093A8
:10152000660180916501882319F085E191E00FC083
:1015300080916601813049F028F0823051F48CEEC0
:1015400090E005C08CE091E002C08CEF90E00E943A
:10155000620480916801823008F462C08091640165
:10156000882309F45DC081508093640160E081119B
:1015700017C08EE095E00E94132602E225E047E0C6
:101580006FE48EE095E00E94892661E08EE095E0B0
:101590000E9413268091670190E00E94710540C06F
:1015A0008EE095E00E94132602E225E047E06FE41A
:1015B0008EE095E00E94892661E08EE095E00E9431
:1015C000132600E521E047E060E58EE095E00E940B
:1015D000612603E521E047E063E58EE095E00E94A7
:1015E00061262091680130E040916701C701B9018F
:1015F0000E94FD326330710514F463E070E001E095
:10160000060F52E2459FC0011124B9010E94FD322C
:1016100047E0460F23E061E58EE095E00E948926D1
:101620006091F301C69EB00111246C507E4F8FE093
:1016300091E00E9493336EE271E08FE091E00E94AE
:10164000883341E06FE071E081E592E00E9444035D
:10165000882309F45ECE81E592E00E94A51460E043
:101660008EE095E00E94132608E029E048E260E061
:101670008EE095E00E94892661E08EE095E00E9470
:1016800013262CE731E048E260E08EE095E00E940E
:1016900031283FCE6091680180916701860F8150AB
:1016A00005C0809167018F5F609168010E94DD3203
:1016B00090936701892F90E00E947105D092640198
:1016C00012CFDF91CF910F91FF90EF90DF90CF90ED
:1016D000BF900895C7E080EC94E00E948B2088239F
:1016E000D1F364E08AEC94E00E946825882341F0FD
:1016F00085EE94E00E94E32D0E9474090E94670722
:1017000043E062E08AEC94E00E947F25882311F197
:101710008091F3018F5F8093F3019091F10189171C
:10172000B8F01092F30180913E0290913F02019631
:1017300090933F0280933E022091400230914102FB
:10174000821793073CF010923F0210923E0202C0B3
:101750000E94A70643E063E08AEC94E00E947F25A4
:10176000882359F18091F3018C5F8093F30190916C
:10177000F101891748F441E065E08AEC94E00E94A9
:101780007F25882309F4A9C08091F3018370809399
:10179000F30180913E0290913F02019690933F02A7
:1017A00080933E02209140023091410282179307BC
:1017B00024F010923F0210923E0243E060E08AEC77
:1017C00094E00E947F25882319F18091F301811113
:1017D0001AC0C093F30180913E0290913F02892B81
:1017E00041F4809140029091410290933F02809396
:1017F0003E0280913E0290913F02019790933F02FA
:1018000080933E0205C081508093F3010E94A70699
:1018100043E061E08AEC94E00E947F25882349F14F
:101820008091F301843048F041E065E08AEC94E077
:101830000E947F25882309F453C08091F3018C5FB7
:101840008093F30180913E0290913F02892B41F4F5
:10185000809140029091410290933F0280933E021A
:1018600080913E0290913F02019790933F028093B6
:101870003E0220913E0230913F0280913C029091C5
:101880003D022817390751F00E94670780913E02F8
:1018900090913F0290933D0280933C0261E08EE084
:1018A00095E00E9413268091310590913205A09118
:1018B0003305B091340587709927AA27BB27049771
:1018C000A105B10528F060E08EE095E00E941326A6
:1018D0008091F3010E949206FECE0E94A7066DCF72
:1018E0008091F30184508093F3010E94A706C1CF39
:1018F000EF92FF920F931F93CF93DF93C0E0D0E05E
:10190000CE010E94C33381110FC02196C11584E01E
:10191000D807B1F786E890E0DF91CF911F910F9142
:10192000FF90EF900C94620464E472E08FE091E029
:101930000E9493336EE271E08FE091E00E94883361
:101940008AE790E00E94620443E46FE071E081E581
:1019500092E00E944403811103C088E690E0DCCF4E
:10196000C0E0D0E009E611E0FE01E956F1407F0158
:10197000F1E0093E1F0749F0C701800F911F0E9447
:10198000C333F80181938F01F3CF40E850E069E65B
:1019900071E081E592E00E943315C058DF4FC11518
:1019A00084E0D807F9F681E592E00E94A5148EE65E
:1019B00090E00E9462048EE095E0DF91CF911F914C
:1019C0000F91FF90EF900C94CB2580EC94E00E9457
:1019D00007241092DD041092DC048CE08093300523
:1019E00066E871E080EC94E00E948B238EE095E045
:1019F0000E94BA2581E0809314051092D80426E84D
:101A000031E04CE060E08EE095E00E94312885E610
:101A100091E00E9451048EE095E00E94CB2524E0E5
:101A20004AE06FEB74E088EB94E00E94D50E8823C7
:101A300009F499C088E994E00E94A51461E081E767
:101A400092E00E94A61E882351F061E772E088E9C7
:101A500094E00E94F610882309F485C008C060E075
:101A600081E792E00E94A61E8111EFCF7CC0809199
:101A70009804807709F477C088E994E090934A0548
:101A800080934905E2E8F7E7E491E0934402E3E854
:101A9000F7E7E491E0934502E4E8F7E7E491E093A7
:101AA0004602E5E8F7E7E491E0934702E6E8F7E766
:101AB000E491E0934802E7E8F7E7E491E093490214
:101AC000E8E8F7E7E491E0934A02E9E8F7E7E49110
:101AD000E0934B02E4E4F2E08081803209F410826A
:101AE000319682E0EC34F807B9F7809144028823FC
:101AF00021F00E94780C0E94CA0361E081E792E025
:101B00000E944D0341E068E974E081E592E00E94A3
:101B1000ED13882391F00E947306882349F0809189
:101B200042029091430201969093430280934202B5
:101B300081E592E00E94A514E5CF20914202309108
:101B40004302C901019797FD079633E09595879564
:101B50003A95E1F7019690934102809340021092EA
:101B600015050C94670781E591E00E9451048EE011
:101B700095E00E94CB25FFCF109211051092100521
:101B80008EE491E090930F0580930E0510927602FB
:101B9000109298041092990489E18093BB041092EA
:101BA000BE048FE391E090937202809371021092D1
:101BB0005102109252021092500210924F0287E38B
:101BC00091E090934E0280934D02089590E022E0C0
:101BD000281740F0892F806A86958CBD909591706A
:101BE0009DBD08959730B0F7220F953010F431E085
:101BF00001C032E0930FECCF8FEF8EBD0DB407FE26
:101C0000FDCF8EB508958EBD0DB407FEFDCF0895AE
:101C100061E0FC0182810E94DB2F8FEF0C94030EA8
:101C2000CF93DF93EC018C810E94E60D60E08A8106
:101C3000DF91CF910C94DB2FCF92DF92EF92FF9246
:101C40000F931F93CF93DF93EC018B017A010E94D6
:101C5000592E6B010E94FC0D8D838F3F49F40E9429
:101C6000592E6C197D096D327140A0F381E103C0DA
:101C70008E3F39F08FE08B83CE010E94080E80E00A
:101C800028C0E114F104E1F081E0E81AF1088FEFD7
:101C90008EBDF8012FEFCF01801B910B8E159F0594
:101CA00038F40DB407FEFDCF8EB52EBD8193F3CF72
:101CB0000DB407FEFDCF8EB5F801EE0DFF1D80833C
:101CC0001D820E94FC0D0E94FC0DCE010E94080E98
:101CD00081E0DF91CF911F910F91FF90EF90DF9006
:101CE000CF9008950F931F93CF93DF93EB010E9442
:101CF000592E8B010E94FC0D8F3F49F00E94592EF6
:101D0000601B710B6C177D07A8F380E001C081E0B8
:101D1000DF91CF911F910F910895FF920F931F9321
:101D2000CF93DF9300D000D0CDB7DEB78C01F62E75
:101D300029833A834B835C830E94100E68E572E02E
:101D4000C8010E94720E8F2D80640E94030E8C8148
:101D50000E94030E8B810E94030E8A810E94030E53
:101D600089810E94030EF11002C085E901C087E855
:101D70000E94030E8CE0F81202C00E94FC0DF12CB0
:101D80000E94FC0DF801858387FF05C0FFEFFF1659
:101D900011F0F394F5CF0F900F900F900F90DF910B
:101DA000CF911F910F91FF900895BF92CF92DF9234
:101DB000EF92FF920F931F93CF93DF93EC01B22E1C
:101DC0001E821B82798368834A830E94592E8B016D
:101DD00061E08A810E94A22F61E08A810E94DB2F4C
:101DE0002A9A229A239A259A80E48C830E94E60DEF
:101DF0002AE0F22E8FEF0E94030EFA94D9F720E02A
:101E000030E0A90160E0CE010E948D0E813049F0E2
:101E10000E94592E601B710B613D774080F381E079
:101E200051C02AEA31E040E050E068E0CE010E9473
:101E30008D0E853011F481E00AC094E0F92E0E94E5
:101E4000FC0D8D83FA94D9F78A3A59F482E08E8397
:101E50008E81823079F4C12CD12CE12C80E4F82ED3
:101E60000CC00E94592E601B710B613D7740C8F277
:101E700082E028C0C12CD12C760120E030E0A901FD
:101E800067E3CE010E948D0EA701960169E2CE01A3
:101E90000E948D0E882349F00E94592E601B710B01
:101EA000613D774050F38AE00DC08E818230E9F4C5
:101EB00020E030E0A9016AE3CE010E948D0E882364
:101EC00039F088E08B83CE010E94080E80E012C0BA
:101ED0000E94FC0D807C803C11F483E08E830E9484
:101EE000FC0D0E94FC0D0E94FC0DCE010E94080E0C
:101EF000BC8281E0DF91CF911F910F91FF90EF9015
:101F0000DF90CF90BF9008950F931F93CF93DF93EF
:101F1000EC0189018E81833039F039E0440F551F7F
:101F2000661F771F3A95D1F79A01AB0161E1CE01A7
:101F30000E948D0E81110AC040E052E0B801CE012E
:101F4000DF91CF911F910F910C941C0E84E08B8335
:101F5000CE010E94080E80E0DF91CF911F910F917A
:101F600008950F931F93CF93DF93EC01862F8A017F
:101F70000E94030EF80180818EBD818122E030E055
:101F80000DB407FEFDCF8EBD2115F2E03F0739F0FD
:101F9000F801E20FF31F80812F5F3F4FF1CF0DB4A7
:101FA00007FEFDCF8FEF0E94030E8FEF0E94030EFE
:101FB0000E94FC0D8D838F71853039F083E18B8316
:101FC000CE010E94080E80E001C081E0DF91CF9138
:101FD0001F910F9108950F931F93CF93DF93EC01FF
:101FE00089018E81833039F089E0440F551F661FC7
:101FF000771F8A95D1F79A01AB0168E1CE010E9463
:102000008D0E882319F086E08B830CC0A8016EEF3B
:10201000CE010E94B10F182F882321F0CE010E941B
:10202000080E04C0CE010E94080E10E0812FDF913F
:10203000CF911F910F910895FC0182818068828366
:102040009F01245F3F4F448555856685778586814E
:1020500097810C94B71D9F92AF92BF92CF92DF925F
:10206000EF92FF920F931F93CF93DF93EC01888140
:1020700085FF02C0912C5EC088899989AA89BB8995
:1020800081159E4FAF41B105A8F7CE010E941C10EB
:10209000982E882379F34C855D856E857F858E81AA
:1020A0009F810E94CE1C6B017C018E819F8125E067
:1020B000B701A60180960E948C1C5C010097D1F2AA
:1020C00080E092E0F5019C01119221503040E1F74F
:1020D00011E0AE81BF8112960C9112971017A0F4F7
:1020E000ED91FC9111970280F381E02D9501B701EC
:1020F000A601410F511D611D711DCD010995882358
:1021000009F4B8CF1F5FE5CF10E020E030E089E0B0
:10211000000F111F221F331F8A95D1F74889598953
:102120006A897B89400F511F621F731F488B598B2F
:102130006A8B7B8B892DDF91CF911F910F91FF903F
:10214000EF90DF90CF90BF90AF909F900895CF9386
:10215000DF93EC01262F4C895D896E897F898E8102
:102160009F8180960E948C1C9C01009761F08C815D
:102170009D818F70992745E0880F991F4A95E1F757
:10218000820F931F02C080E090E0DF91CF9108950D
:10219000CF93DF93DC01FC0190E048E080E05EE259
:1021A00020812032C1F0983031F4EB01C80FD11DED
:1021B00058838F5F40E120813FEB320F3A3130F49A
:1021C0001C963C911C97342309F0205EEB01C80F4C
:1021D000D11D28838F5F9F5F31969B3009F7FB01EC
:1021E000E80FF11D1082DF91CF910895FC018081ED
:1021F000811114C080E2DF01982F1D929A95E9F7B2
:1022000077836683DB0115969C91903119F09032AB
:1022100029F480E4808381E08283089580E008953A
:102220002F923F924F925F926F927F928F929F92E6
:10223000AF92BF92CF92DF92EF92FF920F931F93D4
:10224000CF93DF9300D000D0CDB7DEB79C838B83D4
:102250004B017A01DC018C91882309F112969C9143
:1022600090FF1DC027C0D380D822A114B10409F06B
:102270009CC0D1109AC0452B462B472B09F47EC039
:10228000AB81BC811C964D915D916D917C911F97A6
:1022900029813A81CF010E94E61C87FF7EC0AB8175
:1022A000BC8111968C911197826011968C938FEF5F
:1022B0009FEFE3C083FF17C0EB81FC81808D918D80
:1022C000A28DB38D4089518962897389841B950BD6
:1022D000A60BB70BA70160E070E0481759076A0723
:1022E0007B07D0F018C085FF17C0AB81BC81169664
:1022F000ED91FC9117978681978155E0880F991F82
:102300005A95E1F750962D913C915197821B930B72
:102310008E159F0508F47C018701EB81FC813C96BA
:10232000FA83E983612C42E0742E0115110509F44A
:1023300068C0AB81BC8150964D915D916D917C914F
:1023400053975A01B1E0BB22EB81FC8120810680CA
:10235000F781E02DDB01CA0139E0B695A795979585
:1023600087953A95D1F725FF7ECF448D558D668DA3
:10237000778D480F591F6A1F7B1F2BC026FD02C097
:10238000EB81FC81848D958DA68DB78DEB81FC81D1
:1023900084879587A687B78708C0811106C0EB811F
:1023A000FC818081807769F57ACFAB81BC811C96F6
:1023B0004D915D916D917C911F9716968D919C9199
:1023C00017970E94CE1CAB01BC014D0D511D611D24
:1023D000711DEB81FC8186819781A114B104B1F557
:1023E0000115F2E01F0790F1DC0193962D903D90CE
:1023F0004D905C909697421553056405750529F438
:1024000025C0C701801B910B38C0DC01ED91FC9108
:102410000190F081E02D94010995882309F43FCFC4
:10242000C12CF2E0DF2E8C0C9D1CEB81FC8180899D
:102430009189A289B3898C0D9D1DA11DB11D808B31
:10244000918BA28BB38B0C191D096FCF93012A19A5
:102450003B0968012017310708F4690120E08096E4
:102460000E948C1C009709F41ACFBC016A0D7B1DD9
:10247000A601C4010E947F33D6CF0F900F900F901A
:102480000F90DF91CF911F910F91FF90EF90DF9010
:10249000CF90BF90AF909F908F907F906F905F9004
:1024A0004F903F902F900895FF920F931F93CF93DB
:1024B000DF931F92CDB7DEB78C01262FFC01408938
:1024C000518962897389DB01CA01E5E0B695A79558
:1024D00097958795EA95D1F7F82FFF70FF2E11F0A9
:1024E000211117C041E050E0BE016F5F7F4FC8016E
:1024F0000E941011813019F080E090E01CC0F801BA
:102500004089518962897389415E5F4F6F4F7F4F68
:1025100005C0405E5F4F6F4F7F4FF801408B518B7E
:10252000628B738BF801868197818796F0E2FF9E1C
:10253000800D911D11240F90DF91CF911F910F916C
:10254000FF9008954F925F926F927F928F929F9229
:10255000AF92BF92CF92DF92EF92FF920F931F93B1
:10256000CF93DF93EC016A017B014C845D846E8420
:102570007F84A881AA2309F48CC041155105610507
:10258000710529F41C861D861E861F867CC0A3FF4C
:102590000BC0488D598D6A8D7B8D4C155D056E0580
:1025A0007F0508F476C014C0A5FF12C0EE81FF813C
:1025B00086819781F5E0880F991FFA95E1F7A0E0F1
:1025C000B0E084179507A607B70708F462C05BC0A0
:1025D000088919892A893B89EE81FF81848190E0ED
:1025E0000996B901A8014150510961097109082EE4
:1025F00004C076956795579547950A94D2F746019A
:102600005701B1E08B1A9108A108B10804C0B69433
:10261000A794979487948A95D2F784169506A60670
:10262000B70620F0012B022B032B81F4A6FF05C077
:10263000848D958DA68DB78D04C08C8D9D8DAE8DAE
:10264000BF8D8C879D87AE87BF8704C0841A950A8B
:10265000A60AB70A8E01045F1F4F81149104A104DA
:10266000B10489F04C855D856E857F8598018E81EA
:102670009F810E94E61C91E0891A9108A108B10887
:1026800018165CF306C0C88AD98AEA8AFB8A81E0F8
:1026900005C04C865D866E867F8680E0DF91CF9197
:1026A0001F910F91FF90EF90DF90CF90BF90AF9070
:1026B0009F908F907F906F905F904F9008958F9232
:1026C0009F92AF92BF92FF920F931F93CF93DF938E
:1026D000EC01F22E80E2DE011D928A95E9F7FB0102
:1026E000868197819F838E835D834C83848C958CB8
:1026F000A68CB78C88869986AA86BB86FC01B7967D
:102700004F705527B5E0440F551FBA95E1F7E40F18
:10271000F51F338533FF03C0188280E054C0377142
:1027200038832385287111F4386038830B832F2D6B
:10273000227319F02881217179F72F2D2F702A83A8
:10274000DC0193964D915D916D917C9196974C8BA8
:102750005D8B6E8B7F8B4489558960E070E0BA0198
:1027600055274427028D138D20E030E0402B512B5C
:10277000622B732BF4FE0AC04115510561057105EA
:10278000E9F00E94591E811119C0C6CF4C8F5D8F90
:102790006E8F7F8F448D558D668D778D488F598FC5
:1027A0006A8F7B8FF5FE0EC0488D598D6A8D7B8DAB
:1027B000CE010E94A212811105C0AECF8A8180682D
:1027C0008A83F0CF81E0DF91CF911F910F91FF902D
:1027D000BF90AF909F908F9008958F929F92AF92ED
:1027E000BF92DF92EF92FF920F931F93CF93DF93ED
:1027F0007C01EB01D42EFC018081811138C08881DD
:102800008077A9F1088919892A893B890F711127D5
:1028100022273327012B022B032B49F500E010E080
:1028200088889988AA88BB8860E0CE010E945412EB
:102830000097E9F0FC0120812223C9F02E3211F427
:1028400000E0EECF253EE1F3338533FD07C00023E2
:1028500081F00E94991618130AC00BC03F3081F70F
:1028600026FFDECF022F0F71FC011585D9CF80E046
:102870000EC0B501A40115E076956795579547956B
:102880001A95D1F72D2DBE01C7010E945F13DF916C
:10289000CF911F910F91FF90EF90DF90BF90AF907D
:1028A0009F908F9008950F931F93CF93DF93EC0128
:1028B0008881882309F443C08A8187FF38C061E09A
:1028C000CE010E94A7108C01009729F489818160B4
:1028D000898380E035C0FC018081853EB9F3888121
:1028E00083FF08C0488D598D6A8D7B8D448F558F2D
:1028F000668F778F4C8D5D8D6E8D7F8DF801538F38
:10290000428F758B648BE0914705F09148053097B5
:1029100059F0B8016A5E7F4FC80148960995F801E1
:10292000808D918D938B828B8A818F778A838E8124
:102930009F8180960E94391C882341F201C081E06A
:10294000DF91CF911F910F910895CF93DF93EC0109
:102950000E9453141882DF91CF910895CF92DF9295
:10296000EF92FF920F931F93CF93DF93CDB7DEB714
:10297000E3970FB6F894DEBF0FBECDBF8C017B018D
:102980005BAB4AABD22E19821A82FC01808188236C
:1029900011F080E059C0FB0180818077D1F3EAA972
:1029A000FBA980818F32D9F4EAA9FBA980818F32FB
:1029B00021F43196FBABEAABF7CFF7016681778163
:1029C000811104C0C8010E94F6103EC0CE010196DC
:1029D0000E94F6108823E9F2CE0101967C0150E2B4
:1029E000C52EAE014E5C5F4FBE016F5D7F4F8AA961
:1029F0009BA90E949E17882361F2EAA9FBA9808106
:102A00008823D1F021E0AE014F5D5F4FB701C801CF
:102A10000E94D219882309F4BCCFF801DE01119677
:102A20008C2D01900D928A95E1F7C8010E94A514A2
:102A3000FE0131967F01D5CF2D2DAE014F5D5F4F49
:102A4000B701C8010E94D219E3960FB6F894DEBF11
:102A50000FBECDBFDF91CF911F910F91FF90EF90EF
:102A6000DF90CF9008952F923F924F925F926F9296
:102A70007F928F929F92AF92BF92CF92DF92EF920E
:102A8000FF920F931F93CF93DF93EC015B014A01F9
:102A9000888183FF0EC08A8181FF0BC082FF0FC037
:102AA000488D598D6A8D7B8DCE010E94A2128111B5
:102AB00006C08981816089838FEF9FEF06C1A401E1
:102AC00060E070E088899989AA89BB898095909592
:102AD000A095B09584179507A607B70750F3640132
:102AE0001E012CE0220E311C488959896A897B8994
:102AF000C114D10409F4C7C08E819F812A013B0112
:102B000029E076946794579447942A95D1F7DC018D
:102B100013961C9114217A01B1E0FB22111134C0EB
:102B2000E114F10489F54C855D856E857F8541153D
:102B300051056105710569F091010E94E61C87FD50
:102B4000B8CF811121C0CE010E941C1081111CC080
:102B5000B0CF8C8D9D8DAE8DBF8D0097A105B10539
:102B600079F4CE010E941C10882309F4A2CF8C8531
:102B70009D85AE85BF858C8F9D8FAE8FBF8F04C026
:102B80008C879D87AE87BF874C855D856E857F85E9
:102B90008E819F810E94CE1CAB01BC01410F511D53
:102BA000611D711DEE81FF81E114F10421F4C11456
:102BB00022E0D206B8F580E092E08E199F098601E6
:102BC0008C159D0508F48C01E114F10479F4488812
:102BD00059886A887B88888D998DAA8DBB8D481607
:102BE00059066A067B0610F025E001C021E0CF01FE
:102BF00080960E948C1C009709F45BCFA801B50158
:102C00008E0D9F1D0E947F33E00EF11EE11482E0C5
:102C1000F80641F58E819F8180960E94391C8111B2
:102C200021C047CF83A194A1A5A1B6A18417950780
:102C3000A607B70741F410A28FEF9FEFDC0183A333
:102C400094A3A5A3B6A38E819F81DC01ED91FC9195
:102C50000280F381E02D95010995882309F429CF9D
:102C600000E012E088899989AA89BB89800F911FA9
:102C7000A11DB11D888B998BAA8BBB8BA00EB11E99
:102C8000C01AD10A31CF888D998DAA8DBB8D2A812A
:102C900084179507A607B70728F4488F598F6A8FBE
:102CA0007B8F06C08091470590914805892B11F0D4
:102CB00020682A838A8183FD02C0C40106C0CE0138
:102CC0000E9453148111F9CFF4CEDF91CF911F915F
:102CD0000F91FF90EF90DF90CF90BF90AF909F90BB
:102CE0008F907F906F905F904F903F902F900895BE
:102CF000653040F4FC01E60FF11DE60FF11D818106
:102D0000928108956B3040F4FC01E60FF11DE60F4F
:102D1000F11D848195810895613140F4FC01E60F35
:102D2000F11DE60FF11D86819781089580E090E006
:102D30000895FC0190E080E080FB879587F9219160
:102D4000820F9F5F9B30C1F70895CF93DF93FC0103
:102D5000DB0118964D915D916D917C911B97452BF0
:102D6000462B472B41F416966D917C911797DF9176
:102D7000CF910C94F61080E2EF0119928A95E9F751
:102D800080E1808381E0828316968D919C911797D4
:102D90009783868318964D915D916D917C911B97D9
:102DA000448F558F668F778F81E0DF91CF910895A3
:102DB0002F923F924F925F926F927F928F929F924B
:102DC000AF92BF92CF92DF92EF92FF920F931F9339
:102DD000CF93DF93CDB7DEB7A1970FB6F894DEBFE0
:102DE0000FBECDBF8C016B015A0119821A82FC0102
:102DF0008081811104C0F6011082412C85C04D30C4
:102E00005105C8F3F8018381811106C0B601C801DC
:102E10000E941E1C482E78C0B801CE0101960E9467
:102E2000A516882341F35524539446018A0C9B1C14
:102E300021E0821A9108F80183818515E0F2652C62
:102E4000712CF801448155814619570960E070E002
:102E500085E0440F551F661F771F8A95D1F7CE0175
:102E600001960E94A212482E882329F260E0CE012A
:102E700001960E9454127C01009709F4BCCFFC011A
:102E800083858F3009F0B7CF80818F7190E068160D
:102E9000790609F0B0CFC3010197FDE0F89F30013A
:102EA000F99F700C11241601260C371C50E0652F79
:102EB000C70159A30E94781659A1009791F06A148E
:102EC0007B04D0F42FEF621A720A8F37910510F449
:102ED000282F01C02FE3F10121931F015F5F5D30B7
:102EE00031F76A147B0440F4F701808186FF04C047
:102EF000F601E60DF71D1082F4011082F7018081C2
:102F000086FD02C0539497CF842DA1960FB6F894F6
:102F1000DEBF0FBECDBFDF91CF911F910F91FF900C
:102F2000EF90DF90CF90BF90AF909F908F907F9069
:102F30006F905F904F903F902F900895CF92DF92C7
:102F4000EF92FF920F931F93CF93DF93FB01DC016E
:102F500001962C912032D9F3B483A383ED01BE01F5
:102F60006A1B7B0B8991811105C0CD01860F971FCC
:102F7000EC0118C08F32C9F38C3511F480E0D0C059
:102F8000982F977F9232D1F38A33C1F3982F9F7B8A
:102F90009C33A1F392EC980F923080F380528F35DE
:102FA000F0F2ECCF1C2F3D2F29912032D9F32F3294
:102FB000C9F3EA0118833983EC016115710561F0E9
:102FC0008A918E3211F0803219F461507109F5CF77
:102FD0006F3F710509F094F67283618380E090E0A1
:102FE00020E2EF01C80FD91F2E8301968B30910587
:102FF000C1F7ED01CE018A1B9B0B29912E32D1F333
:103000002032C1F351E0009709F050E09B012150BC
:10301000310938F407E010E0C12CF12CC8E0EC2EA7
:103020000FC0ED01C20FD31F48814E3281F7F2CF9E
:10303000ED01C80FD91F4881403231F450E00196AC
:1030400086179707ACF343C04E3221F4281739078F
:10305000A9F704C04232A1F04C3791F0C6EDC40F7D
:10306000C63010F44D3261F4C6ECC40FC63040F0E7
:10307000C5EAC40FC33020F0CFEDC40FCE3530F019
:103080008217930709F150E04FE503C082179307B9
:10309000D9F00117D0F1CFE9C40FCA3118F440526A
:1030A000FE2805C0CFEBC40FCA3108F4CE28DD24BA
:1030B000D394D10EEF01C10FD11D4E8346E04D15C3
:1030C00008F0D5821D2DBBCF0A30C9F450E08681AF
:1030D000803209F453CF552339F0CF2011F082E02C
:1030E00001C08F2D808309C081E080838581E80F36
:1030F000F11D8EE7868381E3878381E011C0C901DA
:103100000AE018E040E1E42E9ACF0A30F9F22817DD
:103110003907E4F2C9010AE018E050E1E52E8ECF4C
:10312000DF91CF911F910F91FF90EF90DF90CF90A3
:103130000895BF92CF92DF92EF92FF920F931F9369
:10314000CF93DF93CDB7DEB7A0970FB6F894DEBF6D
:103150000FBECDBF8C0119821A82DC018C9183FDD8
:1031600002C080E089C0F801828181FFFACF448DDE
:10317000558D668D778D411551056105710549F0B5
:10318000D80116968D919C9117970E94591E8823FD
:1031900041F361E0C8010E94A7107C01009709F388
:1031A0000E949916D82E85EEF7018083D8011C92D3
:1031B00016968D919C91179780960E94391C8823B2
:1031C00081F2F8019381992309F456C0B801CE0128
:1031D00001960E94A516882321F2BB24B39425EE04
:1031E000C22EF80183818B1508F4BBCFEB2CF12C98
:1031F000D80114964D915C9115974E195F0960E0C6
:1032000070E095E0440F551F661F771F9A95D1F720
:10321000CE0101960E94A212882309F4A2CF60E099
:10322000CE0101960E945412FC01009709F499CF37
:1032300083858F3009F095CF2081822F8F7190E0A8
:10324000E816F90609F08DCF8585D8128ACFC0829D
:10325000D8011696ED91FC91179780A1816080A30B
:1032600026FF08C016968D919C91179780960E9414
:10327000391C02C0B394B5CFA0960FB6F894DEBF48
:103280000FBECDBFDF91CF911F910F91FF90EF90B7
:10329000DF90CF90BF900895AF92BF92CF92DF9210
:1032A000EF92FF920F931F93CF93DF937C01EB017B
:1032B000AD8002E010E07EE7B72E6E0186E0C80E1A
:1032C000D11C89819A819801280F391FEB81FC81DB
:1032D000AF01480F591FE417F50779F0C90165E000
:1032E000880F991F6A95E1F7820F931F2191332769
:1032F00027FD309528273927EECFE3E0EA1510F4B3
:1033000053E0A52E84E08A0D922F9F70E82FF0E005
:103310009A3010F4905D01C0995CEC0FFD1F96830C
:1033200044E0369527954A95E1F78150A81660F359
:10333000FE01EA0DF11DB68240E050E0BA01C7017E
:103340000E94A21261E0C7010E945412BC010097C2
:1033500031F481E0F70191819923C9F017C0FC0194
:103360008081882359F0838583FDECCF4BE050E0CA
:10337000C6010E947233892B29F702C081E007C081
:103380000F5F1F4F0436110509F09BCF80E0DF91DE
:10339000CF911F910F91FF90EF90DF90CF90BF9052
:1033A000AF9008952F923F924F925F926F927F92CB
:1033B0008F929F92AF92BF92CF92DF92EF92FF9245
:1033C0000F931F93CF93DF93CDB7DEB72B970FB635
:1033D000F894DEBF0FBECDBF3C017B876A877A01C0
:1033E0002A83DA0111968D909C901297FB018081BF
:1033F000807711F480E0F3C1D3018C918111FACF71
:10340000FA018081837009F4E1C1C4010C966DE07A
:1034100070E00E94E93255245394560E40E050E08B
:10342000BA018A859B850E94A2121C821D82198284
:10343000412C10E000E01B821701B6E02B0E311C7E
:10344000AA85BB8550962D913D914D915C915397E6
:1034500065E056954795379527956A95D1F75901B7
:1034600061E0CD0128873E8349875F830E94541223
:103470006C0128853E81009739F4EA85FB858181BE
:10348000882309F488C0B6CFDC018C91853E11F009
:1034900081110AC0111102C02C833D83151508F457
:1034A0001F5F811104C077C0151528F005C0853E47
:1034B00019F400E0C5CF10E08E32D9F3F601938500
:1034C0009F3009F046C0011108C086FFB9CF082F10
:1034D0000F7125852983402E07C04A948411E9CFB6
:1034E000858529812813E5CF842D90E00197ADE0F3
:1034F000A89F5001A99FB00C1124A814B904C8F6C4
:1035000020E0622FC60128870E9478162885A8141B
:10351000B90419F4892B69F693CF8F3F910509F00F
:1035200040F63FEB380F3A3108F4805EA5014F5F5B
:103530005F4FD7011396ED91FC911497EA0DFB1D97
:1035400090813FEB390F3A3108F4905E8913B1CF87
:1035500040C193FDAECF002351F0B1E04B124ACFF2
:10356000C6010E9499162981821344CF10C04BE0F6
:1035700050E0B101C6010E947233892B09F060CF7F
:10358000D7018C9180FF03C021E02B8359CF2A8182
:1035900027FF14C12FCF8A818274823409F02ACF89
:1035A000112359F0AC80BD8008C060E08A859B85FE
:1035B0000E945412892B21F01F5F1515B0F318C01B
:1035C000AA85BB8511968C91882391F013CF8A85AB
:1035D0009B850E942B10882309F40CCFAA85BB85FC
:1035E0001696ED91FC9117978281823018F4105F46
:1035F000151568F32B81222341F0B7018A859B853D
:103600000E944C19882309F4F5CEA50160E070E012
:1036100025E0440F551F661F771F2A95D1F78A852D
:103620009B850E94A212882309F4E4CE0FEF050DBA
:10363000102F8FE0482E670186E0C80ED11C9DE058
:10364000592E49C060E08A859B850E9454125C0116
:10365000009709F4CFCEAA85BB851696ED91FC9113
:10366000179780A1816080A3412F101301C040648F
:10367000F501408343861486C60149870E94991646
:10368000D5011D968C931D975B961C921E925A979E
:10369000F7012381348149854F7150E04150510930
:1036A000549EC001559E900D1124F50160E08815CF
:1036B0009905A0F4D901A80FB91F4C91552747FDD2
:1036C00050956530B0F4528341836F5F0196329616
:1036D0006D3069F711501111B5CF13C041E050E0C2
:1036E0008815990511F440E050E051954195510934
:1036F000E8CF6B3018F455834483E7CF5783468374
:10370000E4CFEA85FB8580899189A289B38915E098
:10371000B695A795979587951A95D1F75C0160E0C6
:10372000CF010E9454126C01009709F463CE80E22D
:10373000D6011D928A95E9F7F70136968BE0D601FE
:1037400001900D928A95E1F7F70180818871D60189
:103750001C968C93E0914705F0914805309739F01D
:10376000B601625F7F4FC6014096099509C081E2AC
:1037700098E2F601918B808B80E098E097878687AE
:10378000D60150968D919C91519753969C938E9310
:10379000529759969C938E9358971E968D919C9113
:1037A0001F9757969C938E935697AA85BB8516961E
:1037B000ED91FC91179780A1816080A32A81A501DA
:1037C0006A857B85C3010E945F1309C05524539409
:1037D00025CE2F5F2D3009F433CE5A0192CE2B9691
:1037E0000FB6F894DEBF0FBECDBFDF91CF911F9112
:1037F0000F91FF90EF90DF90CF90BF90AF909F9090
:103800008F907F906F905F904F903F902F90089592
:103810006115710581F0DB010D900020E9F7AD0124
:1038200041505109461B570BDC01ED91FC91028080
:10383000F381E02D099480E090E00895CF93DF9329
:10384000EB01FC012081211102C080E00FC0207635
:1038500021F08FE28883198208C060E00E94A710DF
:10386000009799F3BE010E94C81081E0DF91CF91CB
:103870000895BF92CF92DF92EF92FF920F931F9322
:10388000CF93DF93EC01888180FF39C089819A81D1
:103890008E01095F1F4FDC01ED91FC914B815C8132
:1038A0006D817E810280F381E02D98010995B82E0B
:1038B000811102C0B12C25C0888181FD04C088819E
:1038C0008E7F88831EC0A981BA81ED91FC911197EA
:1038D0001C964D915D916D917C911F97CB80DC8002
:1038E000ED80FE804C0D5D1D6E1D7F1D0280F381FD
:1038F000E02D9801CD0109958111E1CFDBCFBB24EB
:10390000B3948B2DDF91CF911F910F91FF90EF908A
:10391000DF90CF90BF900895CF92DF92EF92FF9209
:103920001F93CF93DF93EC016A017B01122F4B8130
:103930005C816D817E814C155D056E057F0501F111
:103940000E94391C811103C080E090E01FC012FF6B
:1039500006C01882CB82DC82ED82FE8211C0898192
:103960009A81DC01ED91FC910190F081E02D9E01A6
:10397000295F3F4FB701A60109958111EACFE4CF36
:1039800013708881812B8883CE010796DF91CF91B8
:103990001F91FF90EF90DF90CF9008954250510912
:1039A00061097109FC01048004C0440F551F661FA2
:1039B000771F0A94D2F780899189A289B389480F29
:1039C000591F6A1F7B1FCB01BA010895CF92DF9266
:1039D000EF92FF920F931F93CF93DF93EC016A0155
:1039E0007B0189018D81803251F5E7E076956795FD
:1039F00057954795EA95D1F78C899D89AE89BF89FE
:103A0000480F591F6A1F7B1F22E0CE0180960E943B
:103A10008C1C009711F48FEF40C0E894C7F8DD24A8
:103A2000EE24FF24F601EE0FFF1FEE0FFF1FE80F3D
:103A3000F91F40815181628173817F701DC0803187
:103A400051F74C895D896E897F894D0D511D611D2E
:103A5000711D22E0CE0180960E948C1C0097D9F245
:103A6000DD24EE24FF24F601EE0FFF1FE80FF91FFF
:103A70004081518160E070E0888D998DAA8DBB8D69
:103A800084179507A607B70738F0F80140835183DC
:103A90006283738381E001C080E0DF91CF911F9149
:103AA0000F91FF90EF90DF90CF9008958F929F92AB
:103AB000AF92BF92CF92DF92EF92FF920F931F933C
:103AC0006A017B0148015901FC012581203231F551
:103AD00017E076956795579547951A95D1F704891C
:103AE000158926893789400F511F621F731F23E0F4
:103AF00080960E948C1C009799F0E894C7F8DD240A
:103B0000EE24FF24F601EE0FFF1FEE0FFF1FE80F5C
:103B1000F91F80829182A282B3821DC0203111F0F0
:103B200080E01AC0FC0144895589668977894D0D6A
:103B3000511D611D711D23E080960E948C1C009711
:103B400079F3DD24EE24FF24F601EE0FFF1FE80FCA
:103B5000F91F9182808281E01F910F91FF90EF9079
:103B6000DF90CF90BF90AF909F908F9008953F923D
:103B70004F925F926F927F928F929F92AF92BF927D
:103B8000CF92DF92EF92FF920F931F93CF93DF9329
:103B9000CDB7DEB728970FB6F894DEBF0FBECDBF06
:103BA0009E838D832A013B0138872F834115510560
:103BB0006105710531F4FC0180849184A284B38491
:103BC00002C04A015B0175016401FFEFCF1ADF0AF1
:103BD000EF0AFF0AED81FE81808D918DA28DB38D5C
:103BE0008C159D05AE05BF0528F402E0C02ED12C32
:103BF000E12CF12C9E012F5F3F4FB701A6018D8173
:103C00009E810E94E61C87FD1DC0882341F08981AA
:103C10009A81AB81BC81892B8A2B8B2B31F0C81404
:103C2000D904EA04FB0489F60DC00FEF1FEF2FEF54
:103C30003FE0B701A6018D819E810E94561D382E5E
:103C4000811102C0312C1CC0411451046104710463
:103C500059F097018601B301A2018D819E810E94D6
:103C6000561D811107C0EECFED81FE81C086D18641
:103C7000E286F386EF81F885C082D182E282F38208
:103C8000832D28960FB6F894DEBF0FBECDBFDF910F
:103C9000CF911F910F91FF90EF90DF90CF90BF9049
:103CA000AF909F908F907F906F905F904F903F90DC
:103CB00008959F92AF92BF92CF92DF92EF92FF92C0
:103CC0000F931F93CF93DF9300D000D0CDB7DEB713
:103CD0005C016A017B019E012F5F3F4FB701A60186
:103CE000C5010E94E61C982E87FF02C080E01EC01E
:103CF00000E010E09801B701A601C5010E94561D21
:103D00008823A1F3F5014085518562857385C4162A
:103D1000D506E606F70620F4C086D186E286F3864D
:103D2000C980DA80EB80FC809110D5CF0F900F9086
:103D30000F900F90DF91CF911F910F91FF90EF9017
:103D4000DF90CF90BF90AF909F900895CF92DF9279
:103D5000EF92FF920F931F93CF93DF93EC01162FF7
:103D60001D8281E090E0A0E0B0E088879987AA8773
:103D7000BB87DAA3C9A318A28FEF9FEFDC018BA347
:103D80009CA3ADA3BEA3662321F1653008F0BFC09C
:103D900020E040E050E0BA01CE0180960E948C1CE9
:103DA000009709F4B4C0FC0100E1109FE00DF11D83
:103DB0001124E255FE4F80818F7709F0A8C0C0849E
:103DC000D184E284F384C114D104E104F10421F428
:103DD0009EC0C12CD12C760120E0B701A601CE01F6
:103DE00080960E948C1CFC01009709F490C083858A
:103DF00094858115924009F08AC08089823009F04B
:103E000086C086859785892B09F481C035853A83DC
:103E10008FEF830F8B831C8289E090E021E03217C3
:103E200041F0019709F473C0220F4C814F5F4C831E
:103E3000F6CF468957894115510519F060E070E0C9
:103E400004C044A155A166A177A14C875D876E8708
:103E50007F878685978597018601080F191F211D89
:103E6000311D0C8B1D8B2E8B3F8B818992899F83FB
:103E70008E83440F551F661F771F400F511F621F0F
